:020000040000FA
:02000000B02826
:08000800F000030EF100831269
:100010000B11010800000000083E81004E08031982
:100020001628C90AC91C1628CE03C901B80A3808FF
:10003000FA3A031D1D28BE0A6C143E080A3A031D35
:1000400060283808F73A031D6028BE01B8018614FD
:10005000033084262830922633103F1C3328AE1BF1
:1000600033143C1439283F14AE01AF01B001B10183
:10007000B201AE1B60283208FF0703185020310878
:10008000FE07031852203008FD07031854202F08DC
:10009000FC07031856202E08FB0703185820602879
:1000A000FE0F0800FD0F0800FC0F0800FB0F080002
:1000B000FA0F0800F90F0800F80F0800F70A080007
:1000C000B50A3508FA3A031D8B28B501B60F692821
:1000D000B70A371C8B2868303606031D8B283B1C5B
:1000E0007D2886303A06031D7D28A0303906031D81
:1000F0007D28B901BA01BB018B2872080319822837
:10010000F20B842885180614B601B701B90F8B28A5
:10011000BA0F8B28BB0A511085189E280610043090
:10012000F200D21CA9285114861411308326013004
:100130003B275407AC0008308626A928D218A928E6
:10014000511486141130832601303B27AC0008304F
:1001500086260508D200710E8300F00E700E09008D
:1001600007309F000610831608308600F2308500A5
:100170008330810083124C2653103C1406303B27F9
:10018000D40007303B27D5008601F2010530BE00C0
:1001900085011030AD2632308600000005140000C5
:1001A0000510B12606120511000005140000051007
:1001B000B1262C30BA260E30BA260130BA262030AD
:1001C000AD260630BA260130BA262030AD260E30D4
:1001D000BA26061186140A3083265030AC00083047
:1001E00086268614063083260430AD000030AC002D
:1001F000103086265B26851806148B168B1713295C
:100200005008031907295008013A031D0D295118F8
:1002100013293C1C0D2A3C1013295118662A6C1C0A
:100220000D2A6C10662A3B08CC003A08CB0039082E
:10023000CA00CD01E8268030BA260330AA00243057
:10024000840030300002031D2A29A926840AAA0B43
:1002500021292F290008BF26840AAA0B2A29000871
:10026000BF262E30BF262808BF266830BF263F1C79
:1002700046292E08E9002F08EA003008EB00331C5D
:100280004C29E909EA09EB0940144C29AE01AF01F8
:10029000B001B101B20139296908CC006A08CB006C
:1002A0006B08CA00CD01E826401C59292D30BF2615
:1002B0005A29A9260330AA00C00122308400303018
:1002C0000002031D6829A926840AAA0B5F296D294B
:1002D0000008BF26840AAA0B68292508BF262E30ED
:1002E000BF262608BF262708BF265730BF268518F9
:1002F0007E29C030BA265426A9268129C030BA26C4
:10030000A3267808CD007908CC007A08CB007B08BA
:10031000CA00DF26E8264408F03903199629773009
:1003200084008001840A841F912981295008013AA0
:10033000031DE6295508E5003730E70051272B302B
:10034000E70066276408E6006508E7007808E5002E
:100350007908E4007A08E3007B08E2008F27063082
:10036000E8000310E50CE40CE30CE20CE10CE00CFB
:10037000E80BB1296308CD006208CC006108CB000E
:100380006008CA00E8262430BF260330AA002030C7
:10039000840030300002031DD229A926840AAA0B4A
:1003A000C929D7290008BF26840AAA0BD229230805
:1003B000BF262E30BF262408BF262508BF26A32629
:1003C000531C00295030AD26D3010D2A0430AA0059
:1003D0002030840030300002031DF329A926840A4E
:1003E000AA0BEA29F8290008BF26840AAA0BF329D8
:1003F0002408BF262E30BF262508BF262608BF2684
:100400002708BF266B30BF265730BF266830BF266F
:10041000531C00295030AD26D3015118142AF03056
:100420008604A026861D00290F3086050617A02603
:10043000861D2E2A0230AD260F30860506170230A3
:10044000AD26861D2E2A53145814D00A50080A3C93
:100450000318582AD00153183C140029D8010F3032
:1004600086058617A026861D662A8030D7000530AF
:10047000AD260F3086058617A026861D662AD70B67
:10048000372A4C26D00153143C148030BA26A726B4
:100490005230BF264530BF265330BF264530BF26D9
:1004A0005430BF26A326A326A9265030AD26002906
:1004B0005008013A031D5F2A4030CE00662A5008DA
:1004C000023A031D662A4E080319D0015008D900CC
:1004D00003192B2AD90303192B2AD9030319E72B54
:1004E000D9030319BC2CD9030319752DD90303199A
:1004F000422CD9030319872AD9030319C62DD9031E
:1005000003196B2BD9030319012BD0012B2A8B1351
:1005100001303B278B17BD004826861DA22A3D08C7
:10052000373C031C952ABD0A972A3830BD008B132F
:10053000013083169B0083123D0841278B175B26F1
:100540005314AA2A4226861DAA2A3D080319002907
:10055000BD03972A8030BA26A9265330BF264130E2
:10056000BF264730BF26A9264C30BF264530BF26C0
:100570005630BF264530BF264C30BF26A326A726BF
:10058000C030BA268518C92AC030BA265426A326F8
:10059000CD2AC030BA26A326A5263D08E5008B1338
:1005A00009303B278B17E70051270B30E700662700
:1005B0006408CA006508CB00E6262608303A03190D
:1005C000E42A2608BF26E92AA9262708303A031973
:1005D000EC2A2708BF26ED2AA9262808BF26A92627
:1005E0005630BF266F30BF266C30BF267430BF2612
:1005F0007330BF26503058188030AD26D301D80153
:1006000000298B1300303B278B17BD004826861D21
:100610001C2B3D08FE3C031C0F2BBD0A112BFF3089
:10062000BD008B13003083169B0083123D084127C9
:100630008B175B265314262B4226861D262B3D083E
:1006400003190029BD0B112BBD0A112B8030BA26CE
:10065000A9265330BF264130BF264730BF26A926E2
:100660004830BF264130BF264C30BF264630BF261B
:10067000A9264330BF265930BF264330BF264C3011
:10068000BF264530BF265330BF26C030BA26851856
:100690004F2BC030BA265426A926A526532BC0308E
:1006A000BA26A326A5263D08CA00E5262608303A24
:1006B00003195D2B2608BF26622BA9262708303A8E
:1006C0000319652B2708BF26662BA9262808BF26F5
:1006D000A326A726FA2A8B1306303B278B17D400B4
:1006E0004826861D852B5408373C031C792BD40AD9
:1006F0007B2B3830D4008B13063083169B0083127B
:10070000540841278B1753148D2B4226861D8D2BA1
:10071000540803190029D4037B2B8030BA26A9265C
:100720005330BF264130BF264730BF26A926483068
:10073000BF265930BF265330BF265430BF26453020
:10074000BF265230BF264530BF265330BF26493022
:10075000BF265330BF26A926C030BA268518B52B30
:10076000C030BA265426A326B92BC030BA26A326F9
:10077000A5265408E5008B1309303B278B17E700AB
:1007800051270B30E70066276408CA006508CB00D4
:10079000E6262608303A0319D02B2608BF26D52B8B
:1007A000A9262708303A0319D82B2708BF26D92BAA
:1007B000A9262808BF26A9265630BF266F30BF2697
:1007C0006C30BF267430BF267330BF26FA2A8B13D5
:1007D00007303B278B17D5004826861D012C55086E
:1007E000FE3C031CF52BD50AF72BFF30D5008B13ED
:1007F000073083169B008312550841278B1753142B
:10080000092C4226861D092C550803190029D503F9
:10081000F72B8030BA26A9264330BF264530BF26A5
:100820004E30BF265430BF265330BF26A9262F3066
:10083000BF26A9266B30BF265730BF266830BF269B
:10084000A326C030BA26A326A7265508CA00E52647
:100850002608303A03192F2C2608BF26302CA9264B
:100860002708BF262E30BF262808BF26A9264330DA
:10087000BF266530BF266E30BF267430BF2673306A
:10088000BF26FA2A8B1308303B278B17BD0048265A
:10089000861D5E2CBD1A502C3D081E3C031C532C9B
:1008A0003D0A3F39BD008B13083083169B0083122D
:1008B0003D0841278B175B2653146C2C4226861D5E
:1008C0006C2CBD1E682C3D081F39013A03196C2C95
:1008D0003D033F39BD00532C8030BA26A926503045
:1008E000BF264830BF264130BF265330BF26453093
:1008F000BF26A726A326A326C030BA26A326A7264E
:10090000BD1E852C2D30BF26872CA9268A2C3D099B
:10091000013E8B2C3D081F39E500FC30E7005127D4
:100920000310E40DE50DE40DE50DE40DE50D2D30AE
:10093000E70066276408CA006508CB00E62625089C
:10094000303A0319A62C2508BF26AB2CA926260869
:10095000303A0319AE2C2608BF26AF2CA92627084B
:10096000BF262E30BF262808BF26A926E430BF2682
:100970007330BF26A926FA2A8B1302303B27D600F4
:1009800003303B27BD008B174826861DE52CD61962
:10099000D02C5608073A031DD02C3D0A0319D42C3D
:1009A0000130BD070318D60A8B13033083169B0052
:1009B00083123D084127023083169B00831256089C
:1009C00041278B175B265314FE2C4226861DFE2CD6
:1009D000D61DF12C56080739031DF12C3D080319CB
:1009E000FE2C3D08E3005608E400E7010130E60074
:1009F000E3276408D6006308BD00D42C8030BA26F3
:100A00004F30BF264630BF264630BF265330BF2664
:100A10004530BF265430BF26A9262E08E9002F08EE
:100A2000EA003008EB00331C192DE909EA09EB094B
:100A300040146908CC006A08CB006B08CA00CD01DD
:100A4000E826401C262D2D30BF26272DA926C001C3
:100A50000330AA002230840030300002031D352DFF
:100A6000A926840AAA0B2C2D3A2D0008BF26840A39
:100A7000AA0B352D2508BF262E30BF262608BF26F7
:100A80002708BF265730BF26C030BA26A3263C30E1
:100A9000BF26D61D4E2D2D30BF26502DA926562DF2
:100AA000D6093D09013EBD000319D60A560807398B
:100AB000CB003D08CA00E6260330AA00253084009A
:100AC00030300002031D692DA926840AAA0B602D6F
:100AD0006E2D0008BF26840AAA0B692D2808BF26A0
:100AE0003E30BF26A526A726FA2A8B1304303B27C3
:100AF000D60005303B27BD008B174826861D9E2D4E
:100B0000D619892D5608073A031D892D3D0A031968
:100B10008D2D0130BD070318D60A8B1305308316BF
:100B20009B0083123D084127043083169B008312EB
:100B3000560841278B175B265314B72D4226861D76
:100B4000B72DD61DAA2D56080739031DAA2D3D081D
:100B50000319B72D3D08E3005608E400E701013012
:100B6000E600E3276408D6006308BD008D2D8030C1
:100B7000BA26A9265030BF264F30BF265730BF2691
:100B80004530BF265230BF26A9260D2D8B130130CC
:100B90003B27BD0009303B278B17D6004826861D12
:100BA000E32D5608963C031CD72DD60AD92D973035
:100BB000D6008B13093083169B00831256084127F9
:100BC0008B175314EB2D4226861DEB2D5608031967
:100BD0000029D603D92D8030BA26A9265330BF2646
:100BE0004130BF264730BF26A9264C30BF264530AE
:100BF000BF265630BF264530BF264C30BF26A9261B
:100C00004330BF264130BF264C30BF26A726C03018
:100C1000BA268518102EC030BA265426A326142EC4
:100C2000C030BA26A326A5263D08E5008B1309305F
:100C30003B278B17E70051270B30E7006627640836
:100C4000CA006508CB00E6262608303A03192B2E89
:100C50002608BF26302EA9262708303A0319332E3E
:100C60002708BF26342EA9262808BF26A9265630D5
:100C7000BF266F30BF266C30BF267430BF2673305E
:100C8000BF26FA2A0F30860586160230AD260800E8
:100C90000F3086050616452E203084008001840A18
:100CA000841F4E2E511408005330BF264130BF26FA
:100CB0004730BF26080086140C30832608307E2675
:100CC00086140F30832600307E268614113083264A
:100CD00001307E2686140B30832604303B27AC007F
:100CE0000530792686140D30832602303B27AC0070
:100CF00003303B27AD001030862608003B27AC00B0
:100D00000830862608008038AC000830AB0086101A
:100D10008511AD0DAC0D0318851506150611AB0B2D
:100D2000882E0800AB00061506110310051A0314DF
:100D3000B20DB10DB00DAF0DAE0DAB0B932E080083
:100D40000000000008002030BF262030BF262030E1
:100D5000BF262030BF2608000F30A900B126A90BFE
:100D6000AE2E0A30AA00A030AB00AB0BB52EAA0BFA
:100D7000B32E0800CC260511D4260511C42ECC268E
:100D80000515D42605150000051400000510643073
:100D9000B400B40BC92E0800C20006080F39860043
:100DA0004208F03986040800000005140000051010
:100DB00006080F398600420EF03986040800031039
:100DC000CA0DCB0DCC0DCD0D0800CB01CC01CD0152
:100DD00003102030C300C401C501C601C701C8010A
:100DE000CA0DCB0DCC0DCD0DC80DC70DC60DC50D53
:100DF000C40DC30B202F44080F393038A000450E16
:100E00000F393038A10045080F393038A200460E9E
:100E10000F393038A30046080F393038A400470E88
:100E20000F393038A50047080F393038A600480E72
:100E30000F393038A70048080F393038A8000800AB
:100E40004830840030274730840030274630840003
:100E50003027453084003027443084003027F02E7E
:100E600003300007CF00CF19800030300007CF00DB
:100E7000CF1B8000080083169B001C141A088312E5
:100E8000080083169A008B131C1555309D00AA305C
:100E90009D009C148B171C119C184C2F9C138312C3
:100EA0000800E4010830E8006508E70C03185C2F2F
:100EB000E80B552FE50100340310612FE70C0318F0
:100EC000E507E50CE40CE80B5E2F0800DA010830BA
:100ED000E800650DDA0D6708DA020318712FDA07EA
:100EE0000310E50DE80B692FDB010830E800640D05
:100EF000DA0DDB0D6708DA02E2010301031C620F61
:100F0000DB0203188B2F6708DA07E20103010318DD
:100F1000620FDB070310E40DE80B772F0800E101F7
:100F2000E0016508DF006408DE006308DD00620898
:100F3000DC000830E800E60C0318AD2FE80B9B2F0F
:100F4000E800E70C0318AB2FE80BA12FE501E40143
:100F5000E301E20100340310DA2F0310C02FE60C86
:100F6000031CC02F5C08E2075D0803185D0FE30750
:100F70005E0803185E0FE4075F0803185F0FE507BC
:100F8000E50CE40CE30CE20CE10CE80BAF2F0830AD
:100F9000E800E70C031CDA2F5C08E2075D08031881
:100FA0005D0FE3075E0803185E0FE4075F08031890
:100FB0005F0FE507E50CE40CE30CE20CE10CE00C40
:100FC000E80BC92F0800EB276608E3070318E40ABB
:100FD0006708E4070800E609E60A0319E703E709DA
:020FE000080007
:02400E00613F10
:1042000064000000000007000D00A800000064002A
:0442100000003B006F
:00000001FF
